:100000003EC04BC04AC0B1C148C047C046C045C051
:1000100075C143C05AC05BC05CC05FC060C063C0F4
:1000200064C067C034C13BC142C149C14EC155C162
:100030005AC1F000F000F0000F000F000F814224C1
:1000400018183C7EFFFF8142241824428180C06042
:1000500030180C060301000103060C183060C08044
:10006000FE1028448200800082FE8200800002028E
:10007000FE02820080000202FE0282008000112443
:100080001FBECFE9CDBF20E0A0E6B0E001C01D92C9
:10009000A237B207E1F7AED1B1C1B2CF85B5816069
:1000A00085BDC49ABC980895E82F87B3807F87BB2D
:1000B00088B3807F88BB8E2F90E088309105E0F474
:1000C000FC01E65FFF4F87B3099483600FC0836034
:1000D00001C0866087BBC19A0895866001C08C60AC
:1000E00087BBC29A08958C6005C0896087BBC09A9F
:1000F0000895896087BBC39A0895EF92FF920F938A
:100100001F93CF93DF937C0100E010E00E151F05D5
:10011000B1F0C0E0D0E02091610030E08C2F0C2ED7
:1001200002C0359527950A94E2F720FF8FEFBCDFD8
:100130002196C830D10579F70F5F1F4FE7CFDF91C8
:10014000CF911F910F91FF90EF90089580916000E3
:10015000ABDF84E690E02ED18FEFA6DF84E690E05F
:1001600029C18F929F92AF92BF92CF92DF92EF926E
:10017000FF921F93CF93DF93C0906200D0906300F3
:10018000E0906400F09065008090660090906700B9
:10019000A0906800B0906900C818D908EA08FB0868
:1001A000A0E0B0E0C816D906EA06FB0600F16A0135
:1001B000162FF22EE9019C2F9F19911728F5809197
:1001C000620090916300A0916400B09165008093FB
:1001D000660090936700A0936800B0936900FE01E9
:1001E000849180936100C60188DF2196E4CF8FEF70
:1001F000DF91CF911F91FF90EF90DF90CF90BF9054
:10020000AF909F908F9050CFDF91CF911F91FF9033
:10021000EF90DF90CF90BF90AF909F908F90089518
:10022000B4991FC0809160008F5F873018F480936D
:10023000600002C0109260001092610087DF86DFCC
:1002400085DF8091620090916300A0916400B0917D
:1002500065008093660090936700A0936800B09358
:100260006900089570D0609362007093630080937A
:10027000640090936500D4DFE09160008E2F90E0E1
:1002800087309105C8F5FC01EE5EFF4F09942DE41F
:1002900030E040ED57E063E18CEA9DE007C02DE4DB
:1002A00030E048EE53E063E180E090E05ACF20E692
:1002B00030E040E450E06DE180E991E0F7CF26E4E2
:1002C00030E040ED57E067E005C02DE330E040ED61
:1002D00057E069E084EC99E0E9CF22E330E048EEB2
:1002E00053E06BE0E1CF80ED97E007DF80916100A4
:1002F0008F5F8093610008958FEFD6CE1F920F928B
:100300000FB60F9211248F939F93AF93BF93809159
:100310006E0090916F00A0917000B09171000196F5
:10032000A11DB11D80936E0090936F00A09370008B
:10033000B0937100BF91AF919F918F910F900FBEBD
:100340000F901F90189580916E0090916F00A09172
:100350007000B0917100BC01CD0124E0660F771FE1
:10036000881F991F2A95D1F708951F920F920FB6F3
:100370000F9211248F939F93AF93BF9380916A0044
:1003800090916B00A0916C00B0916D000196A11D41
:10039000B11D80936A0090936B00A0936C00B093A2
:1003A0006D00BF91AF919F918F910F900FBE0F90F5
:1003B0001F901895009741F0EFE5F9E03197F1F7BC
:1003C00000C000000197F6CF089583B7826083BF15
:1003D0008FB583608FBDF894A89580E481BD789433
:1003E00089B7826089BF12BE789417B886B18768D2
:1003F00086B90895EADF52DE35DFFECFF894FFCFED
:00000001FF
